:020000020000FC
:100000007ACE00000000000020C0C1C18EC00000F8
:10001000000098C000000000000000000203040679
:10002000080C10182030406080000406080C1018DE
:100030002030406080A0C0000003070F1F000D0D9E
:100040000403060D0503030202004FB662FD0CC057
:10005000552041F00994C52DC095089483FDC7959E
:10006000C4BD64604FBE1895C0916400089483FDC0
:10007000C795C4BD6B7FC0916400CF3F09F41EC01B
:1000800070FF1AC082FD05C04FBEC1989798959821
:10009000189576FD0EC064FD0CC0C091B100C0FD86
:1000A0009298C1FD9398C2FD9498CAEFC095CA95E5
:1000B000F1F7C198979895984FBE189524BCCC2716
:1000C000C064C8BF6460F8CFC6CF70FFC4CF64FD02
:1000D000C2CFC19AC0CF70FFBECF64FDBCCF979A8C
:1000E000BACF70FFB8CF64FDB6CF959AB4CF929ACD
:1000F00070FFB1CF64FDAFCFC7E0CA95F1F7C19AE9
:10010000AACF939A70FFA7CF64FDA5CFC7E0CA9589
:10011000F1F7979AA0CF949A70FF9DCF64FD9BCF83
:10012000C7E0CA95F1F7959A96CF4FB6C9B7CF7E7B
:10013000C9BF6E7FCCB5CE0DDDB5DF1DDBBDCABD41
:100140004FBE18953FB68F7EA9B7A072A2118061ED
:10015000A9B7AF7DA9BFA9B7AE7FA9BF7894A09179
:100160006800AA2341F085FD2FC0A0916800AA95E0
:10017000A093680029C040E050E085FD15C0A6B3FB
:1001800096FDA095A0FD4FEFAEB5A06496FDAF7BA8
:10019000AEBDAA27A062A8BF8D7FA6B396FDA0958D
:1001A000A0FD5FEF451739F7A0E461FDA09368005B
:1001B00085FD03C0A0E4A093680040939600816091
:1001C000442311F02092990085FD0EC0A091690092
:1001D000AA2331F0A0916900AA95A093690004C0F8
:1001E0008061AA27A062A8BF80FF0AC0A0919600E4
:1001F0004A2F61FF8E7F85FD01C000C040936100E2
:100200004091B400443009F004C0A0916100A09373
:100210006300A0916000A395A093600059F0F8944A
:10022000A9B7A160A9BF84FF03C0A9B7A062A9BFF5
:100230003FBE1895A0917400A395A093740042E06E
:1002400050916800552329F085FF03C05A955093BB
:100250006800A0919600A13018F0209299000DC07E
:1002600020929A002092A300A0919900AF5FA093E2
:10027000990018F0AFEFA0939900B09061005091F1
:10028000B400523049F465FF91F0A2E3BA1678F059
:10029000A0918600A0936100533049F465FF39F0C6
:1002A000A2E3BA1620F0A091C000A0936100509183
:1002B00062005B1521F010F05A9501C053955093E0
:1002C00062004A95D1F65091A300539509F45A95CE
:1002D0005093A300A091A400AA95A093A40009F0B4
:1002E0004BC0A1E0A093A40048E0A091A500AA23E0
:1002F00081F145E0A091A5005A17F0F1A091A60068
:100300005A1728F441E0A3E0A093A40007C0A091ED
:10031000A7005A1718F441E04093A400D0909C0025
:10032000C0906300DC14A8F0A091B400A430D9F010
:1003300065FD0FC0C0929C00539521F0A091A500CF
:10034000A093A300A1E0A093A400ACE3A09362005B
:1003500013C0A0919C00A40F20F45FEF50939C0069
:1003600002C0A0939C00A0919C00AF3F29F4AFEF86
:10037000A0939A00A093A300F894A9B7A160A9BF85
:1003800084FF03C0A9B7A062A9BF3FBE18953FB6BE
:1003900046B557B58F7EA9B7A072A2118061A9B7E3
:1003A000AF7DA9BFA9B7AE7FA9BF789481FD25C055
:1003B000AEB5AF7B96FDA064AEBD8260A6B396FDE0
:1003C000A095A0FF05C040936500509366001FC133
:1003D000AEB5A06496FDAF7BAEBDAA27A062A8BF54
:1003E0008D7F85FF01C006C140E0A6B396FDA095B4
:1003F000A0FD00C140939600EFC0AEB5A06496FD8D
:10040000AF7BAEBD8D7F61FF72C0AEB5AF7B96FD99
:10041000A064AEBDAA27A062A8BF826040939100ED
:1004200050939200A0908F004A19B09090005B0901
:10043000BB24A22C4C38520518F42092950049C0D8
:10044000A091D400AA2359F1483C520528F4A0E118
:10045000BA2EAAE0AA2E23C04836A1E05A0728F4F3
:10046000A8E0BA2EAFE0AA2E1AC0403DA2E05A077B
:1004700028F4A4E0BA2EAEE1AA2E11C0403AA5E0BD
:100480005A0728F4A2E0BA2EACE3AA2E08C04839D5
:10049000A8E05A0720F4A1E0BA2EA8E7AA2EC42E9D
:1004A000A0919300CA1AD52EA0919400DA0ADD20FB
:1004B0002AF4AFEFC094D094CA1ADA0A20929500B9
:1004C000A8E0A210A0E0CA14DA0618F4A1E0A093F4
:1004D0009500409393005093940040919100509167
:1004E000920040938F005093900042E075C0A0911D
:1004F00065004A1BA09166005A0B94FD60C093FDF5
:100500005EC092FD5AC086FF03C0D52EC42E0CC01B
:100510005695479591FD51C05695479590FD4DC014
:10052000D52EC42ED694C79461FD19C0AC2DAC5104
:10053000AD2DA24008F005C0DD2089F4AC2DA85CEB
:1005400070F4A0916700A395AA2311F0A09367000F
:10055000AA3008F44FC02092960081604BC0A09151
:100560006700AA2319F0AA95A0936700A22C5091C6
:10057000BA0097FD02C0A090C800AAEFAA0EA22D53
:10058000A21DCA18DA0A4FB74170442319F040E09F
:1005900050E015C0AFEFCA16D20418F04FEF50E08C
:1005A0000EC0A091AC00CA9E412D000C441F50E02B
:1005B00008F012C04FEF50E00FC05695479594FFDA
:1005C00007C0552309F04FEFA42FA6954A0F521DDF
:1005D0004F3F520508F04FEF40939600816061FF56
:1005E00009C0AFE1A095A923AB299A2F8F7DBB202D
:1005F00009F48062A0E4A093680085FF03C0AAE02C
:10060000A093680061FD03C085FD01C08F7E85FD5C
:1006100003C0A0E2A0936900F894A9B7A160A9BFA4
:1006200084FF03C0A9B7A062A9BF3FBE189511E01F
:100630000AC013E008C01AE006C01EE104C014E6B8
:1006400002C018EC00C005E1BB27BA95F1F70A9586
:10065000D9F71A95C1F708952AE338E709C020E3CE
:100660003CE806C02AE234EB03C025E238EC00C0C7
:10067000B091AD00BA9509F4089512E0BB27939AA2
:10068000BA95F1F7979ABA95F1F79798BA95F1F765
:100690009398BA95F1F7123009F0C19A123009F423
:1006A000959AB091AD00BA95F1F7123009F0C19862
:1006B000123009F49598B7E8BA95F1F71A95F1F662
:1006C000022FB22FBA95F1F70A95D9F73A9581F62C
:1006D000939A0895221B39E0001F3A9509F4089572
:1006E000221F211B18F4210F8894F6CF0894F4CF11
:1006F000622C722CB0E08894B395221F331FE0F770
:10070000379527958894912E802E020B130B10F4A9
:10071000192D082D10F4889401C00894661C771CCC
:10072000BA9571F7172D062D0895322D11232AF44D
:100730003A9500951095031B130BF894029F712CAA
:10074000002D129F912C802C7894780C172D921CE0
:10075000292DB4E06B2E2695179507956A94D9F745
:10076000332321F000951095031B130B089500917E
:10077000B400043009F474C0B0919600B95198F0F7
:10078000B72FB67081F465FD2BC005E09090C600D0
:10079000B92DBA9521F00AE0BA9509F002E1B091BD
:1007A0007B00B01BE0F065FF0AC0B0919E00B093E3
:1007B0009C00BFEFB093A300B1E0B093A400B09150
:1007C0006100B093630020927E0020927F0020920F
:1007D000800020928100209282006F7D41C0606283
:1007E0009090C600B92DBA9579F4B0916200B09599
:1007F000BB1FBB1F1B2FB7950B2FB12FB170B3952C
:100800001B2FB02FBE7F25C0B92DBA95BA9581F4A4
:10081000B0916200B095BB1FBB1FBB1F1B2FB795CC
:100820000B2FB12FB370B3951B2FB02FBC7F14C00B
:10083000B0916200B095BB1FBB1FBB1FBB1F1B2F1E
:10084000B7950B2FB12FB770B395B3951B2FB02F62
:10085000B87FB0540B2F120900937E0010937F00D5
:10086000089510917B00169500917A000795B0913C
:100870007E00B01B0B2FB0917F00B10B1B2F28F413
:100880000038BFEF1B0740F009C00F37120508F40E
:1008900005C00FE710E002C000E81FEF00938300DF
:1008A00010938400089500918300B09180000B0F95
:1008B00010918400B09181001B1F20E030918400D2
:1008C00033230AF42A95B09182002B1F1AF4203F9B
:1008D00040F00AC02F3008F407C00FEF1FEF2FE0E1
:1008E00003C000E010E020EF30916300B0919B0066
:1008F0003B1718F4323030F009C0B0918400BB23AC
:100900005AF004C0B0918400BB2332F400938000FD
:10091000109381002093820008952091D7000091C8
:100920008300000F10918400111FFFDE11232AF4B1
:100930000038BFEF1B0740F009C00F37120508F45D
:1009400005C00FE710E002C000E81FEF002352F0DF
:10095000B0916200B01B0B2F18F0013008F00AC0F4
:1009600001E008C000950F5FB09162000B0F08F026
:1009700001C00FEF0093850008952091D8000091E9
:10098000810010918200D1DE11232AF40130BFEFE3
:100990001B0740F009C00F3F120508F405C00FEF18
:1009A00010E002C001E01FEF112352F0B09185006A
:1009B000B01B0B2F18F0013008F00AC001E008C08E
:1009C00000950F5FB09185000B0F08F001C00FEF8D
:1009D0000093630008950FEF71FD1EC0B091D30026
:1009E000BB23D1F0B0917B00BB23B1F00FEF10918E
:1009F0007B0070DEF894B091730072FDB5E00B9F40
:100A0000112D002D7894112309F00FEFB0919E0065
:100A10000B1710F400919E0000939D000895009123
:100A20007A0010917B0000541140B0919D0010F4A9
:100A3000BA9501C0B39511F0B0939D000895EBD322
:100A4000B2E074FDB1E0B7B9B6B1B068B064B6B9A0
:100A5000EEDDB2E074FDB1E0B7B9B6B1B068B06434
:100A6000B6B9B6B1B6FDFDCF04B115B1B6B1BF7719
:100A7000B6B928D42CE62093A800222309F441C05B
:100A800030E03093A900732E7694622E6694620E45
:100A9000731E262D372D0217130778F08090A800BB
:100AA000BCE6B80DB093A8008090A900B0E0B81DD6
:100AB000B093A900260D371DEECF8090A80090902E
:100AC000A9001091A90016950091A8000795169508
:100AD000079523E0169507952A95E1F72091B50033
:100AE0002A9529F42092A8002092A9000AC02A95EC
:100AF00021F0800E911E2A95E1F78092A800909235
:100B0000A90008952091B500B6B1B6FDFBCF04B1A0
:100B100015B1B6B1BF77B6B9B091AA00B395B0938D
:100B2000AA00B83060F12092AA00B091D200BB2395
:100B300021F1112329F0B091AB00BF3F61F009C052
:100B4000B091AB000B1739F020F4BB2321F0BA951C
:100B500002C0B395E1F300919B00B093AB00BA3FA4
:100B600050F400ECB93F38F400E8B83F20F400E45A
:100B7000B73F08F400E000939B007F7E089521308A
:100B8000B1F00F3FB3E01B0790F4BCE6BB2379F054
:100B9000B091A8000B17B091A9001B0740F4B091C9
:100BA0009B00BB2359F0BA95B0939B0007C0B0914E
:100BB0009B00BF3F19F0B395B0939B0000919B0041
:100BC000B0916300B01B10F400916300B0919C00E1
:100BD0000B1750F000919C00B0919C00BF3F21F09A
:100BE000B0919C00B0939B00502E00936400B09194
:100BF000AA00B73009F47061089502E3F894B09147
:100C0000D9000B9F012D000C001F7894B0919B0020
:100C10000B1710F000919B0000936100009363009C
:100C2000502E0093640000939E00089520927A0055
:100C3000B0EFB0937B000895F8940CB51DB52091EA
:100C40007400789430917500609076000093750080
:100C500010937600031B160971FD03C077FD80C059
:100C600028C070907700209377002709222319F07D
:100C70000FEF1FEF0EC080907800909079003093B6
:100C80007800609279000091750010917600081943
:100C9000190920917A0030917B0036952795020F33
:100CA000131F10F40FEF1FEF00937A0010937B00D7
:100CB0002BC020917A0030917B003901B4E08B2E5B
:100CC000B2E09B2E343040F08A949A94383020F071
:100CD00072FD02C08A949A94769467948A94E1F79C
:100CE00026193709992021F0169507959A94E1F76E
:100CF000200F311F20937A0030937B0028F43FEFC0
:100D000030937A0030937B00323008F4706871FFC2
:100D100002C0B3E00DC0B091C40000917100023870
:100D200038F0B395003A08F0B395B63008F0B5E066
:100D30009B2EB4E08B2E10917B0000917A0024E072
:100D4000169507952A95E1F70819120928F0B02F92
:100D5000B250B12FB20910F402E010E0980126C0A1
:100D600020917A0030917B003901769467946694E3
:100D7000669466942619320906950695200F321D51
:100D800020937A0030937B00323008F07F7704E0C4
:100D9000369527953695279526952695201B10F094
:100DA000223008F422E089019090C40060FDFECF5B
:100DB000E0908B00F0908C006160B9B7B061B9BF72
:100DC000380177FD41C07694679400938B001093AF
:100DD0008C00B92DB330E1F0B0FD04C0060D171D35
:100DE000930106C0000F111F0250120922E030E0EB
:100DF000B92DB33068F020938D0030938E000093AE
:100E00008700109388006092890070928A003AC02F
:100E100000938D0010938E002093870030938800FC
:100E20006092890070928A0071FF0DC0BFE0B0939C
:100E30008D0020928E00B093890020928A00B0939A
:100E40008B0020928C001EC0669400938B00B92DFD
:100E5000B33091F0B0FD03C0060D262D03C0000F86
:100E6000025022E0B92DB33038F020938D0000936A
:100E700087006092890006C000938D002093870050
:100E80006092890000917C0002FD0350013029F43A
:100E900095FD0AC0B0E0B7B909C0023019F4B7E057
:100EA000B7B904C095FDF6CFB6E0B7B90091A2007E
:100EB000000F10F4BBE60B270093A20060FDFECFED
:100EC000B2E0B0936E006160B9B7B061B9BFB72F3F
:100ED000B670D1F020917A0030917B00369527953D
:100EE0003695279571FF02C0B0E43B0FF8940CB51E
:100EF0001DB5020F131F1BBD0ABD6160B0E1B8BF75
:100F0000B9B7B061B9BF78940895686020927D0048
:100F100020E066FD20E206C0686020927D0020E2AD
:100F200066FD20E001E011E077FD11C0B72FB6703B
:100F300009F0677F14E100917B00069509F40395A1
:100F40000F3008F00FE071FF02C004E114E160FD12
:100F50000FC0B0917D00BB2359F071FF06C0B09166
:100F60006E00BA95B0936E0011F470624FC0ABDFA3
:100F7000B0B7B77FB0BFB8B1B0B7B860B0BFB091CD
:100F80007D00B395B0937D00B8B177FD06C0B1E0A8
:100F900071FDB3E0BA95F1F7B8B1B072B21709F0CC
:100FA0002AC071FF05C00395011708F00A95CFCF3D
:100FB00063FD05C00395011708F0B4CFC8CF677F64
:100FC000F8943CB56DB470907A00B0917B00770CCA
:100FD000BB1F08F4BFEF770CBB1F08F4BFEF370D42
:100FE0006B1E6BBC3ABD6160B0E1B8BFB9B7B06110
:100FF000B9BF789497CFB0916D00B13008F492CF1B
:1010000063FD90CF0A9509F0A2CF7F7D20918D00DE
:1010100030918E00F894B0E1B8BF0CB51DB5020F49
:10102000131F1BBD0ABDE0908700F090880061602F
:10103000B9B7B061B9BF7894B72FB67039F0B09135
:101040006D0072FFB395B0936D0009C075FF07C0C6
:1010500066FD05C063FD03C0BF91BF91F7C408954D
:1010600000E063FF01C001E0F89410917100B7E067
:101070001B9F212D102D7894200F269517952695CE
:1010800017952695179510937100183718F4B8E73F
:10109000B093710000917100B09172000B1720F0B5
:1010A0006061C1989798959860FDFECFE0908900A7
:1010B000F0908A006160B9B7B061B9BF0895B2E03D
:1010C00095FD0AC0F894B0937C00939A929862FFC1
:1010D00001C0959A7894F4C0F894B0937C00939AE8
:1010E000949862FF01C0C19A7894EAC0B3E082FF8D
:1010F00024C095FD11C002E0F894B0937C00E1E8B3
:10110000F0E00093B1009598949A62FF02C0979A1C
:1011100001C093987894D4C002E0F894B0937C0016
:10112000E1E8F0E00093B100C198929A62FF02C03A
:10113000979A01C093987894C3C095FD0BC0F8941A
:10114000B0937C00EBE6F0E0959862FF01C0979ABF
:101150007894B6C0F894B0937C00EBE6F0E0C198C8
:1011600062FF01C0979A7894ABC0B4E095FD0AC0C5
:10117000F894B0937C00929A949862FF01C0979A79
:1011800078949EC0F894B0937C00949A929862FFF1
:1011900001C0979A789494C0B5E082FF24C095FD71
:1011A00011C001E0F894B0937C00E7E7F0E0009311
:1011B000B1009798939A62FF02C0C19A01C09298B9
:1011C00078947EC004E0F894B0937C00EBE8F0E003
:1011D0000093B1009798939A62FF02C0959A01C05C
:1011E000949878946DC095FD0BC0F894B0937C00F2
:1011F000E5E6F0E0979862FF01C0C19A789460C07C
:10120000F894B0937C00E1E7F0E0979862FF01C0AA
:10121000959A789455C0B6E095FD0AC0F894B093BD
:101220007C00949A939862FF01C0C19A789448C058
:10123000F894B0937C00929A939862FF01C0959ABB
:1012400078943EC0B1E082FF24C095FD11C004E057
:10125000F894B0937C00EBE8F0E00093B100C19803
:10126000929A62FF02C0959A01C09498789428C01F
:1012700001E0F894B0937C00E7E7F0E00093B10060
:101280009598949A62FF02C0C19A01C0929878948E
:1012900017C095FD0BC0F894B0937C00E1E7F0E037
:1012A000C19862FF01C0959A78940AC0F894B093EF
:1012B0007C00E5E6F0E0959862FF01C0C19A789461
:1012C0006F7E089524E630E0F9012092B100C198C4
:1012D00097989598929A939A949A6B7F0895A2EB17
:1012E000B0E007E00D9307E00D9301E00D9304E0FB
:1012F0000D930FEF0D930D930AE00D9302E00D9304
:1013000001E00D9301E00D93AEEBB0E001E00D9331
:1013100000E00D9304EB0D930FEF0D930D930D93E0
:1013200003E00D930FEF0D9301E00D930FEF0D937D
:1013300005E20D9300ED0D9308E70D9308EC0D9376
:1013400004E00D930FEF0D9301E00D9300E00D937A
:101350000AE70D930AE00D9300E00D9301E00D9371
:1013600000E00D930FEF0D9300E00D930895209191
:10137000B9008B7F233009F48460B091BA009F7D5F
:10138000B1FD90629F7BB091BB00B1FD90642230B3
:1013900011F0886001C0877F08950A95E00FF21D63
:1013A000B4910895ECE1F0E00091B200F6DFB09363
:1013B000D700ECE1F0E00091B300EFDFB093D8008C
:1013C000EAE2F0E00091B800E8DFB093D9000091C4
:1013D000D100002319F42092A50013C0013108F0B8
:1013E00001E1B02FB00FB00FB093A5001B2FB10FCC
:1013F000B10FB00FB093A600B10FB00FB00FB09304
:10140000A7000091B800023008F402E000937300D6
:10141000B091CE000FEFB23009F400EAB33009F416
:1014200002E800937200E8E3F0E00091D500B5DF38
:10143000B093A000089508952091C8003091C9008C
:10144000B091BA00B33009F43E5097FF02C020E0DB
:101450003FEFB32FB21B6B2EB25810F4B2E86B2ED5
:1014600000E00395609EB12DBD57D8F30093AC000A
:1014700008959068E1DFE1D8E0D820E030E0B0E105
:101480006B2ED7D8B09196002B0F321D6A94C9F7F6
:10149000B4E036952795BA95E1F7822E9F77CCDF99
:1014A0000895F894E3E0F0E0B9E0B7BFB491B07804
:1014B000C1F3F894A895B1B5B861B1BDB0E0B1BDC4
:1014C000B4E0BEBFBFE5BDBFFDDEB0E0B8BBB2E17A
:1014D000B7BBB0E0B5BBB0E0B4BBBCE1B2BBBCEBEA
:1014E000B1BB2224A0E0B0E02D92AA31E9F7A0E63A
:1014F000B0E00FEF2D920A95E9F7B1E0B093A200AA
:10150000EEDEE1D2B6B1B460B6B90091CA00009384
:10151000AD00B1E0B0936A00F89493D89DD88DD80F
:101520009ED88BD89FD889D85DD38BD88AD887D8B6
:10153000F8940AEF1AEFA6B396FDA095A0FF1FC07E
:101540001A95C9F70A95B1F7E0E0FCE1B591B43E10
:1015500039F4B591B03E21F4B591BF3F09F40CC008
:10156000E0E0F395F395B591B83F49F4B591B439FE
:1015700031F4B591BA3A19F4EE27F6950994F7DEED
:1015800011DF59DF59DF0091CA000093AD009ADEE8
:10159000B2E0B3BFB2E0BEBDB2E0B5BDB1E5B8BF29
:1015A000B9BFB0B7B77FB0BFB8B1B0B7B860B0BF60
:1015B0003ED8789444DA20927000BEB5B06496FDAF
:1015C000BF7BBEBDB9B7B062B9BFBB27B062B8BF01
:1015D0008D7F37D8626033E02CE0B0919500BB235B
:1015E00021F42CE03A9509F4A3CF27D880FFA0CFAF
:1015F0008E7FB0919600B23078F3B92FBF71009111
:10160000980000939700B0939800B01729F72A9597
:1016100021F76D7FBEB5B06496FDBF7BBEBDBB2715
:10162000B062B8BF8D7FB091D400BB2321F480623B
:10163000B92FB0709B2F8F7B2092670000D885FF59
:1016400005C0B0916700BA3008F08064F2D702E0BC
:1016500085FF01C000E0B0919600B017B8F3F89490
:10166000FBD7FAD7F9D77894ECD720928600E1D748
:10167000B091BE00B13008F478C0B0916A00B130CA
:1016800008F473C085FD18C0B0919600BF3F08F400
:101690006CC0F894EAD77894D2D7B0919600B13064
:1016A000C0F7F894D9D7C7D7D7D77894C8D7B0910F
:1016B0009600BF3FB0F3C8C2B8E09B2E9068F89484
:1016C000BBDE7894BCD7F8949F77B6DE8090960006
:1016D000B0919600BF37789408F44FC0A8D7F8941B
:1016E000C4D778949A9451F7C4DEB82DB550B0930E
:1016F000C900A7D7F8947BD27894BAE09B2E906863
:10170000F8949ADE78949BD7F8949F7795DE809032
:101710009600B0919600BF37789478F788D7F89400
:101720009BD789D799D778949A9449F7A2DEB82D98
:10173000BB5FB093C8000B2F1091C900125810F076
:10174000100B20F4B2E80B0F0093C9007AD7F8947D
:10175000E7D15CD2789473D7F8946EDE7894B09128
:101760009600BF3F08F48ECF6FC200919600B091F3
:1017700086000B1710F00093860061D701E0B0914E
:10178000BA00B35009F405E0B0919600B01708F024
:101790006ECFF8946AD769D768D7789452D72092D9
:1017A0006A0020926B0020926C00B0916B00B395A0
:1017B000B0936B00BF3F71F5B0916C00B395B093DF
:1017C0006C00B091CC0009E1BA9559F002E3BA95EA
:1017D00041F00DE7BA9529F00AEFBA9511F0209281
:1017E0006C00B0916C00B017A8F06CDD20D7B09100
:1017F0006C00BA95B0936C0020926B00B091CB0056
:10180000B093AD00F89431D77894B091CA00B093FA
:10181000AD0015D710D7B0916800BB2319F485FF30
:1018200001C086CE01E085FD01C006E0B0919600C2
:10183000B01708F4BACF03D7B0916800BB2309F4FE
:1018400077CEF8943FDD20926100209262002092D2
:101850006300522C209264002092A1007894B091F1
:10186000B700BB0FB0939F0020927E0020927F00B4
:101870002092800020928100209282002092AA0073
:1018800060E070E020927100B8E0B093AA0070614F
:10189000CED6B2E074FDB1E0B7B9B6B1B068B0640D
:1018A000B6B9B6B1B6FDFDCF04B115B1B6B1BF77CB
:1018B000B6B9112309F00FEF0093AB0023D9B8E0BC
:1018C000B093AA00706153DDF894BFEFB0939B0012
:1018D00094D9B0916100B0939B00B0939C00B093F9
:1018E0009D007894B1E0B0936100B09363005B2EEB
:1018F000B0936400B093A400B0919A00B093A30099
:10190000B091BA00B33019F49F7D87FD9062716089
:10191000726020926D007FDC95DC88D98DD986D9E4
:101920008BD984D9F9DA23D79BDBC9DB85D9EDDAEA
:1019300065FD97D777FF4FD877FD71D891DBD6DB60
:101940007BD9EADA65FDAFD78BDB0FDC75D9DDDA41
:1019500065FDE3D785DB20DC6FD9DEDA65FD0DD8C8
:101960007FDB59DC69D9D1DAB2E074FDB1E0B7B9F7
:10197000B6B1B068B064B6B973DB64DC5DD9C2D807
:1019800071FF1EC0B0919E00B0939B00B0939C006D
:10199000B0919A00B093A300B1E0B093A40018E115
:1019A0002CE0B0916D00B11728F07D7F746020931A
:1019B0006F0006C0B0919600B13008F0B3CF50C0B0
:1019C00072FF15C066FD13C0B0916F00BA9519F48F
:1019D0007B7F7860A7CFB0936F00B0919600B13055
:1019E00008F0A0CFB091BA00B33009F039C020920E
:1019F0007000B0919900B13058F0B0919E00B09352
:101A00009C00B0919A00B093A300B1E0B093A40001
:101A1000B09199000AEF1091D600112309F003E06C
:101A2000B01708F01DC085FF04C0B0916800BB234B
:101A3000B9F000EF66FF05C0B0919E00B0939B0027
:101A400000E2B0917B00B01708F46CCFB091700049
:101A5000B395B0937000B0919600BB2309F002C01B
:101A600020927000F8942EDC8090B900B2E0B09320
:101A7000B9007DDC8092B900209261002092620062
:101A800020926300522C2092640020929F0060E01C
:101A900070E07894D4D516DC0091D600002319F0BC
:101AA000C19A979A959AB6B1B460B6B985FF05C048
:101AB000B0916800BB2309F43BCDB091BF00B130B9
:101AC00008F0C4CD6ECEEDE0F0E023D0053A09F089
:101AD0001BC0EEE0F0E01DD00A3509F015C03AE079
:101AE000A2EBB0E0E3E0F0E014D00D9331963A952C
:101AF000D9F739E1AEEBB0E0EFE0F0E00AD00D93BA
:101B000031963A95D9F702C0EADB0AD0E8E2F0E074
:101B10000895E199FECFEEBBFFBBE09A0DB30895A7
:101B20001ED03AE0A2EBB0E0E3E0F0E00D910FD080
:101B300031963A95D9F739E1AEEBB0E0EFE0F0E05D
:101B40000D9105D031963A95D9F712D00895E199C3
:101B5000FECF0DBBEEBBFFBBE29AE19A0895EDE02C
:101B6000F0E00FEFF4DFEEE0F0E00FEFF0DF0895CC
:101B7000EDE0F0E005EAEBDFEEE0F0E00AE5E7DFBC
:101B800008953091AE000091AF00313011F4009310
:101B9000B200323011F40093B300333011F40093EB
:101BA000B400343011F40093C600353011F40093C2
:101BB000B500363011F40093B800373011F40093BB
:101BC000C400383011F40093B900393011F4009397
:101BD000CE003A3011F40093BA003B3011F4009378
:101BE000BB00089525E02DD52A95E9F7089534D551
:101BF00036D538D53AD51FD52FD531D533D535D5AE
:101C00001AD52AD52CD52ED530D508952ED52AD53E
:101C100026D522D510D529D525D521D51DD50BD52D
:101C200024D520D51CD518D508958090AE0090906D
:101C3000AF0012D511D510D5FED48A94D1F715D5A1
:101C4000FAD49A94E1F70895F894D1DF7894CADF32
:101C5000C9DFB1E0B093AE00B1E0B093AF00209225
:101C6000B000F894E2DF7894B5E06B2E70909600A7
:101C7000E8D4B09196007B16C9F7B13018F0BF3F99
:101C800040F107C07EDFF8944BDFB1DFB8E0B1BDB3
:101C9000A9DF6A9459F7B091B000B395B093B00042
:101CA000B33008F4DECF9EDFB091AF00B395B093B0
:101CB000AF00F894B091AE00BA95EEE3F0E0EB0F10
:101CC000F21D049178940395B091AF00B01708F419
:101CD000C6CF88DF87DFB091AE00B395B093AE007A
:101CE000B091AE00BC3008F4B7CFF9DAF89418DF41
:081CF000B8E0B1BD77DFD5CBF0
:00000001FF
